S1048000007B
S123C000C779C75BC782C7B6C761C769C771C7C4C7DCC7D4C7E4C836C82CC820C825C83F22
S123C020C857C8A5C867C877C887C92DC94DC959C96DC77FCA50C983C998C98DCAACCAB8F4
S123C040CAC3C9B5C9A1C9BFC9C9C9D9CA1ACA46CA55CA71CA80CA8FCA26CA36CA0BC9F13B
S123C060CAD8CADCCAE2CAF3CB06CAF9CB3CCB0ECB4CCBAFCBC4CBD2CBE4CB87CB91CB6A48
S123C080CB9AD7C0D76CD796D7AED7D3D7E6D7F8D803D81BD840D850D7F1D86BD87FD88A63
S123C0A0D860D895D8A0D8ABD8BDD8CBD8D9D77BD901D926D911D8E7DD38DE16DE1ADE5FE1
S111C0C0DAD4CB9DCBA6DAADDAE3DAF40000D5
S123C500FCFF0227318E00FFBDE1131AB3FF022608CC0000FDFF02201DBDDBC8CEC529BDA8
S123C520DD27B6700027FB20134D454D4F5259204641554C54008EFEFF7F003C8D33B670D7
S123C5400084038103260D8E00FF0FBDE113FDFF027EE0AFB6700027037EC704B680004A28
S123C56026F7CC8001CEC300ED008600A7097EC704CE002A4FA700088C003926F8CE100099
S123C5801C2608863EA7097F00227F0023CC07C0DD261C39801D282086B0A72B860CA72D58
S123C5A086059739BDDBC8CC0000DD0CDD12DD148608970BCCC110DD16DD18DD1A8620B71E
S123C5C0C6EACEC300C6208640A7098FC300108F5A26F6CEC300DF08CCC200ED00CCFE0096
S123C5E0ED04C30001ED02830100ED06860AA7088620A709EF0CEF0EDC0CC30001DD0CED0D
S123C6000ABDDAF4CEC62BA6002706BDDB9A0820F6CE10001C200118CE3000180926FC1D0E
S123C62020011D0008CC0000DD2639496E74657261637469766520432020205620322E3859
S123C6403120392F32382F39330A008D6B8D74816125F881732604863E2068368D513C1844
S123C660388D4C328172270D8177270F816327118162271B39A6008D4A2010188FE7002049
S123C6800A188FA400A700EA00E700863E2034188F373C32331B331B97015D270C8D19A754
S123C6A0009B019701085A26F496018D1620DC8D07368D0416328F39B6102E842027F9B6B7
S123C6C0102F39F6102EC48027F9B7102F39DE08A608970A1AEE00EE0218E600F7C6E31834
S123C6E008FCC000FDC6E8BDFFFF20ED8620B7C6EADC088FED021AEF00A60981402604EEFF
S123C7000CDF0839963C260CCE10001F2E2005BDC64B20F0120B02ECDE08EE0EDF088CC394
S123C720002607DC1EC30001DD1EA609810026D4BDC6CE810027CD814027C981202704861C
S123C74002200286048D0220BB9701940B910126013996019A0B970B7EC6C3EC02A30020FE
S123C7601CEC02A400E4012014EC02AA00EA01200CEC02A800E8012004EC00E302ED0208D4
S123C78008398D26A601E6033DDD00A600E6033DDB00D700EC013DDB00D7007D00072706EC
S123C7A04F5F930020D7DC0020D37F00078D6308088D5F090939BDC7AAEC023CEE0002DF8A
S123C7C0003820D7EC00A3022705CC000020AECC000120A9EC02A3002EF520EEEC02A300E6
S123C7E02DED20E63CEC002B1C26043808083937368605B7C7F9EC02380027030926FA38DB
S123C8000808ED00394F5FA30037368604B7C7F920E46D002A094F5FA300ED00730007398A
S123C82063006301394F5FA300ED0039EC002705CC0001ED0039EC0027F64F5FED0039ECA9
S123C84002E306DD00E601E905A600A904ED04DC00ED06C6043A39EC06A302DD00E605E2A6
S123C86001A604A20020E6EC06A302E605E201A604A2002D1E2025EC02A306E601E205A615
S123C88000A2042D0E2015EC06A302260FEC04A3002609C6063ACC0001ED0039C6063ACC25
S123C8A00000ED00397F0007BDC9433CC6043ABDC943CE0000DF0038A603E6073DDD02A6B9
S123C8C003E6063DD301DD01960089009700A602E6073DD301DD01960089009700A603E6F7
S123C8E0053DD300DD00A602E6063DD300DD00A601E6073DD300DD00EC033DDB00D700A6BC
S123C90002E6053DDB00D700A601E6063DDB00D700A600E6073DDB00D700C6043ADC02ED64
S123C92002DC00ED007D000727028D0139CC0000A302DD00C600E2018600A200ED00DC00CC
S123C940ED02396D002A058DE47300073918EC00180818080909ED003918EC020909ED006A
S123C96018EC00180818081808180820E718E600183A18A60009A70018095A26F518E600D6
S123C980183A393CCDEE00E600384F20C38FCDEE00EE028F0909ED008FCDEE00EE008F2012
S123C9A0AF18E6003C3AEC00DD00EC02380909ED00DC00209D18E6003C3AEC003820933C42
S123C9C0A601CDEE00A70020083CEC00CDEE00ED0018083818080808393CEC00DD00EC029E
S123C9E0CDEE00ED02DC00ED0038C6043A57183A39EC00DD00EC02D70718E6003C3AD607BC
S123CA00ED02DC00ED0038080820C9EC00D70118E6003C3AD601ED0020B9A6013CEE02275A
S123CA203FA70038202AA601B7CA323CEE0227301C00FF38201AA601B7CA423CEE02272043
S123CA401D00FF38200AEC003CEE022713ED00380808080839EC00DD00EC023CEE04260673
S123CA603886057EDE6BED02DC00ED0038080820DFEC003CEE0227E8E70038ED02080839AB
S123CA80EC003CEE0227D9ED0038ED02080839EC00DD00EC023CEE0427C6ED02DC00ED0093
S123CAA038EC02ED04DC00ED020808393CEE0027AFE6004F38ED00393CEE0027A3EC00389C
S123CAC0ED00393CEE002798EC00DD00EC02380909ED02DC00ED003918EE00391AEE000802
S123CAE00839EC00260618EE0008083918081808080839EC0026EF20F3EC0027EFCC00011E
S123CB00ED0018EE0039EC0026E218EE0039EC00DD0018EC00DF04D3048F1AEE002705DC8C
S123CB2000ED0039DE088640A7098621B7C6EAEC0C1AEE0E8FCDEF0C1AEF0E3918EC00DFC9
S123CB4000D3008F1AEE0027DB080839EC00DD00EC02DD0218EC00DF04D3048F1AEE022708
S123CB60C3DC00ED00DC02ED0239DF00DE08DC00A306CDA300250718081808DE00391809C1
S123CB80DE0086047EDE6B8F18E3008F18081808393C323318E3007EC950EE0039EC00DDAD
S123CBA03A0808180839DC3A0909ED00180839EC003CEE021AA300382427E302C30002ED71
S123CBC002080839EC003CEE021AA3003824120520E8EC003CEE021AA30038240405052057
S123CBE0D97EDE65EC003CEE021AA3003824F218A60018083D20C33CBDD6DCCE00003CDFE2
S123CC003DDF3F7F00411830CDEE06A600BDCD4F2528812D260B73004108A600BDCD4F25E1
S123CC2019812E260B08A600BDCD4F24037ECCBD3131BDD6E638860F0D39A600BDCD4F24B1
S123CC4077BDCCCE0824F37C003DA60008BDCD4F25F5812E260AA600BDCD4F24030820F6E6
S123CC6081452707816527037ECD1108A600BDCD4F2515812D2706812B270520B31863008E
S123CC8008A600BDCD4F24A8803018A70108A600BDCD4F241418E601585818EB0158803053
S123CCA01B18A701088126228718A601186D002A01409B3D973D2059812E26A408A600BD85
S123CCC0CD4F249C8D0808258D7A003D20EF963E9743DC3FDD440579003E252C0579003EAC
S123CCE02526D34436963E9943973E32251A0579003EDD3F2512E600C0304FD33FDD3F96AA
S123CD003E89002503973E39DC44DD3F9643973E39CDEF06CE003DBDCD7A272C963D18A739
S123CD20018696973DBDCD5B186D01271B2A0BCECD85BDD70F1860012006CECD89BDD70FF3
S123CD40BDCD99186A0126F83131BDD6E6383981302506813922020D390C39CE003D8D1AC8
S123CD6027147D003E2B0FDC3F7A003D270A0579003E2AF5DD3F0C390D393736EC00260279
S123CD80EC023233393DCCCCCD41200000BDD035BDD6DCBDCF04BDD6E67D003D27057D0063
S123CDA042260ACC00009741DD3DDD3F39964198469741963D9B422A0924168606CEFFFFE8
S123CDC02009250D8607CE0000DF40DF3DDF3F0D398B82973DCE00003C3C30BDCE126D0099
S123CDE02B0B69036902690169007A003D6D032A13A6024CA702260CC601E3002404467C88
S123CE00003DED0038DF3E329740317D003D27B45F399645D6403DA7019644D6403DE30042
S123CE20ED009645D63F3DE300A70324026C026F006F019643D6403DE302ED029644D63FE5
S123CE403DE302ED0224026C019645D63E3DE302ED0224026C019643D63F3DE301ED012476
S123CE60026C009644D63E3DE301ED0124026C009643D63E3DE300ED0039BDD6DCCED40865
S123CE80BDD70F7D00412703730046BDCF36BDD6E64FD63DC17F24035F201B53C3FF902FD8
S123CEA0178FDC3E2001040926FC7D00412A074353C300012A020C3986090D39CC0000DD26
S123CEC0004FD63DC17F24035F203353C3FFA02F2F8F96405FDD00DC3E20070476000076EE
S123CEE000010926F67D00412A147300007300014353DE0008DF002605C300012A020C396A
S123CF0086090D39BDD370CE0045964280972A1BC6038B082A096F00095A26F66F0039C606
S123CF20804A2B035720FAE400E7008D028D07964688FF974639963D260EDC42DD3DDC44BE
S123CF40DD3F964697415F397D004227F9D641D84690422510811822ED183C36CE004318EF
S123CF60CE003E201740811822D0183C369642973D96469741CE003E18CE004317363636C7
S123CF80A8003617A8013617A8023630A606E7061684074CC4185454543AE6034A27095641
S123CFA066026601660020F45618A602A900974018A601A901973F18A600A902973E30A63B
S123CFC0062B15245A76003E76003F7600407C003D264CCCCDBB2053251B730041700040D4
S123CFE024087C003F26037C003E70003F24037C003E70003E7D003E2B252613963D800886
S123D0002326973DDC3F27207F0040DD3E20E67A003D271478004079003F79003E2AF01A60
S123D020EE07C6093A355F39CCCDC41AEE07ED07C6073A3539CE0042BDCD7A260486080D73
S123D04039CE003DBDCD7A26020C39BDD6DC964698419741CE00003C3C3C86183630DC3E7B
S123D0601A934326049640914524107C0042261986060D38383831BDD6E639DC3F9344DDC2
S123D0803F963E9243973E6A00740043760044760045963DD642501B2B062506860720D307
S123D0A025CE8B7F973DDC3EED049640A706DC3F9344DD3F963E9243973E2A08EC04DD3E44
S123D0C0A606974069036902690178004079003F79003E6A0026CF630163026303DC3F9325
S123D0E044963E9243EC0224030C2003C30001DD3FA6018900973E241176003E76003F7602
S123D10000407C003D26037ED0700C7ED0733CCE003DBDCD7A260738CC3000ED0039DE3D71
S123D1203CDE3F3C964136BDD6DCCE00003C3C3C1830CDEE0F86207D004127057F00418670
S123D1402DA70008CDEF00CED278BDD70FBDD27C2E19CED274BDD70FBDD27C2E16186A029C
S123D160CECD89BDD70FBDCD9920DC186C02CECD8520F0CED408BDD70FBDCF36D63DC07FAE
S123D18050CB17200A74003E76003F7600405A26F4860118A70318A6028B082B0A81082420
S123D1A0064A18A7038602800218A702186D032E15862ECDEE00A70008186D03270586303B
S123D1C0A70008CDEF00CED25F860718A705186F04DC3FA301DD3F963EA200973E2505189D
S123D1E06C0420EDDC3FE301DD3F963EA900973E18A6048B303CCDEE00A70008186A032673
S123D20005862EA70008CDEF0038080808186A0526BCCDEE0009A600813027F90818E602EA
S123D220272A8645A70008862BA7005D2A0550862DA70008CDEF004FCE000A02378FCB30E3
S123D240CDEE00E7000833CB30E700086F00383838BDD6E632974138DF3F38DF3D38390F3F
S123D26042400186A00027100003E800006400000A000001497423FE4B18967F96462A1202
S123D280D6412A0EDC421A933D2617DC441A933F20109141260CDC3D1A93422605DC3F1A4E
S123D2A093440784F424028A080639CE008EC3000026057ECDC409052AFCDD3E7F00408F27
S123D2C09741D73D5F394D2AE24353C30001CEFF8E20DBCE009EC30000261118DE00260338
S123D2E07ECDC40978000179000059492AF5DD3E960097408F9741D73D5F394D2AD5730005
S123D300007300014353DE0008DF002603C30001CEFF9E20C1CE003DBDCD7A2601397D0015
S123D320412A04860A0D39BDD6DC860436DE3F3CDE3D3C18308D399642807E4C2A03442004
S123D34003448B7E9742BDD035BDCF367A003D8D1F18EC00DD3D18EC02DD3F186A0426E6E7
S123D360DC42DD3DDC44DD3F383831BDD6E65F39DC3DDD42DC3FDD449641974639BDD6DCB3
S123D380CED4D7BDD70FBDD035BDD6E6DC3D1A8385B32B0B7D004126037ECDBB7ECDC4BD55
S123D3A0D6DC9641367F0041BDCF04DC4227068086544C26FC5C37CED3ECBDD69CCED3E86F
S123D3C0BDD70F2003BDCD99306A0026F832324D2A0CBDD370CED630BDD6F6BDD035BDD60F
S123D3E0E65F39BDD6DC20EA402DF8543638EF1D37D00D0139500D013AB60B613C088889A2
S123D4003D2AAAAB3E2AAAAB3F0000003F8000003F800000FFBDD431BDCD997ED38C8D1173
S123D420BDD6DCCED4D7BDD70FBDCD99BDD6E65F3996412704860C0D39963D27F8BDD6DCEE
S123D4403C3C30BDD7274FD63DC07F2A0143BDD2C6CED4D3BDD70FBDCD9930BDD70FBDD75F
S123D46027867F97423C3C30BDD735CED630BDD6F6BDCF3630BDD70FBDD727CED4CFBDD681
S123D480F6BDCF3630BDD70FBDD03530BDD727BDD370BDCD99CED4B2BDD69C30BDD70FBD1A
S123D4A0CD99383830BDD70FBDCF363838BDD6E65F393E1D89D93E3A2E8C3E638E393E9255
S123D4C049253ECCCCCD3F2AAAAB40000000FFBF8000003F3172183EDE5BD9860E0D398651
S123D4E00D0D39BDD6DC9641367F0041CED630BDD70FBDD27C2F07BDD3E386FF20014F3643
S123D5003C3C30BDD727BDD370BDCD99CED53ABDD69C30BDD70FBDCD993838324D270CCE8F
S123D520D536BDD70F730041BDCF36BDD686329741BDD6E65F393FC90FDBBCE2DD1B3D705A
S123D540F0F1BD8888893D9D89D9BDBA2E8C3DE38E39BE1249253E4CCCCDBEAAAAAB3F805F
S123D5600000FFBDD6DC4F2005BDD6DC86F036CED64EBDD70F2003BDCF36964126F9200317
S123D580BDCF2BBDD27C2EF88D61240930A6002B04880FA7008D54240930A6002A04880F98
S123D5A0A7008D47240730A60088F0A700CED694BDD70FBDCD99BDD370BDCD993C3C30BD46
S123D5C0D735A6042A05CED6352003CED620BDD69C30A6044724037300414D2B06BDD70F56
S123D5E0BDCD99383831BDD6E65F397A0042BDD27C2E020C397C0042730041BDCF367A0068
S123D600420D39BDCF04DC3DDE42DD42DF3DDC3FDE44DD44DF3F9641D6469746D7415F397E
S123D6203638EF1DB9500D013C088889BE2AAAAB3F800000FF37D00D01BAB60B613D2AAA03
S123D640ABBF0000003F800000FF40490FDB43B40000BDD6DCBDD370BDD569BDD606BDD59F
S123D66063BDD0352407BDD6E6860B0D39BDD6E65F397FFFFFFFBDD6DCCED694BDD70FBD72
S123D680CD99BDD6E639BDD6DCCED69820EECED64A7ED6F63C8EFA3142652EE18FDE3D3CEC
S123D6A0DE3F3C8F9641363CCC0000DD3DDD3FDD40201030A6029746EC03DD44EC05DD4211
S123D6C0BDCD9930EE00BDD70FBDCF3638C6043A3CA6004326DD30C6073A3539383C3C8F58
S123D6E03037367ED735300808BDD70F38313131316E00CED6307F0041EC02DD3FEC000523
S123D7002403730041973D27020D56D73E5F397F0046EC02DD44EC0005240373004697429F
S123D72027020D56D74339DC3FED02DC3D58D1414656ED0039DC44ED02DC4258D14646567F
S123D740ED00397F00415F397D003E2705CC7F80DD3D4F5FDD3F397D003E27037300415F80
S123D76039BDD70F08080808BDD6F6393C183CEC00BDD2C6183838090920AC3C183C080810
S123D780BDD6F60909EE00BDD10E183838EC00ED0408080808393C183CBDD6F6BDCEBC182A
S123D7A0383824037EDE6BED00DC00ED02393C183CEC02DD00EC00BDD2FB1838387ED72741
S123D7C03C183CBDD6F6BDCE9118383824037EDE6B205D3C183CBDD761BDCF361838380846
S123D7E00808087ED7273C183CBDD761BDCF2B20EBA6008880A700393C183CBDD761BDCDAD
S123D8009920093C183CBDD761BDD03518383824037EDE6B080808087ED7273C183CBDD7C5
S123D82061BDD27C183838260CCC0001080808080808ED00390808080808086F006F013953
S123D8403C183CBDD761BDD27C1838382BDB20E53C183CBDD761BDD27C1838382ECB20D59B
S123D8603C183CBDD761BDD41520A13C183CBDD6F6BDD31518383824037EDE6B7ED7273CCC
S123D880183CBDD6F6BDD38C20EA3C183CBDD6F6BDD37D20DF3C183CBDD6F6BDD43120D48D
S123D8A03C183CBDD6F6BDD41E20C93C183CBDD6F6BDD4E30736BDD676320620B73C183C41
S123D8C0BDD6F6BDD686BDD56320A93C183CBDD6F6BDD686BDD569209B3C183CBDD6F6BD26
S123D8E0D686BDD652208D8602E6019D47080839BDDBE0A600BDDCC4A601BDDCC4080820EB
S123D90003BDDBE0A600BDDCC4A601BDDCC4080839BDDBE03CEE008602E60027059D470810
S123D92020F738080839183CDF00BDDB401A830051240C8621B7C6EADE001838180939DEAE
S123D94000DC00C30002E300DD02830002DD04DE02EE000808A60026037EDA9B812527038A
S123D9607EDA8908A6008166261BDF02DE0409093CBDD6F6380909DF04CEC100BDD10ECE2C
S123D980C1007EDA7B8164267DDF0218CEC100DE040909DF04EC022A0C862D18A700180852
S123D9A0CC0000A302CE000A02378FCE000A02378FCE000A02378FCE000A02378FCE000A9A
S123D9C00237183C388601335D27064FCB30E70008334D27045D27064FCB30E70008334D13
S123D9E027045D27064FCB30E70008334D27045D27064FCB30E7000833CB30E700085FE764
S123DA0000CEC10020758178262ADF02DE040909DF04A602BDDCAABDDB88257217BDDB8804
S123DA20256CA603BDDCAABDDB88256217BDDB88255C206181632611DF02DE040909DF04B2
S123DA40A603BDDB882547204C8162261EDF02DE040909DF04E60318CE00085886308900D4
S123DA60BDDB882529180926F2202A8173261ADF02DE040909DF04EE020808A6002708BD33
S123DA80DB88250A0820F4200CBDDB882409860ABDDB9A2006DE02087ED955DE00DC00C362
S123DAA00002E3008FCC0000ED001838393CDC14C300011A931426FBC30001CE0000081A26
S123DAC0931426FA8F380909ED00CC000C0909ED007EC782090909090FDC14ED02DC120E09
S123DAE0ED0039EC0008083C183CEE00AD00183838ED00390F3C183CB6103C84402605CEC9
S123DB00FF002003CEBF003CC6C03A18CEE1251AEF0008083C32324D26F538CCC500EDFE95
S123DB20CCDEE5EDE2CCDED8EDE0CE10006F226F248630A7211C23181C22181838380E3938
S123DB40960B84082707CC00F0DD062016DC1893162307830001DD062009CC00F09316D302
S123DB6018DD06960B84102705CC00F02012DC1A931623058300012007CC00F09316D31A93
S123DB801A93062302DC06393736BDDB401A83000224040D323339322001370F3CDE160806
S123DBA08CC2002603CEC110DF16A700960B840827119C18260DDE18088CC2002603CEC15F
S123DBC010DF1838330C0E398D79CC00389D47C60C9D478D198601970F8608971C4F971DC1
S123DBE0CC00019D47C6069D47C68F9D4739CC00409D478602CEDC03E6009D47088CDC43AC
S123DC0026F639000A1F1F0E04000000001111110F010E00000000000C040800000F1111B7
S123DC200F010E00000C0C000C0C0000000C0C000C0408020006020202120C00000A0E041A
S123DC40000000CEDC5818CE0047A60018A7000818088CDCAA26F339FF0096CE10000F1D01
S123DC603C201D0010B700986F078104260F8601B710041C0010A6031D001020228601B7C4
S123DC8010041C0010A6031D0010848026EF86FFA707B60098A704E7031C00101D00101CC6
S123DCA03C20FE00960E3900000036840F8B30813A2B028B071632444444448B30813A2B32
S123DCC0028B0739BDDCAA371686029D47339D4739CE000A02378FCE000A02378FCE000A0F
S123DCE002378FCE000A02378FCE000A02379D47CC00019D47CC00079D47CC008F9D478696
S123DD000233CB309D4733CB309D47C62E9D4733CB309D4733CB309D4733CB309D47C66D98
S123DD209D47C6739D4739CC00029D478602E60027059D470820F739183CDF00CC7FFFDDC3
S123DD4004CEC3001AEE0E188CC3002607CCE400DD06200518EC04DD06EC0693063CDE0038
S123DD60A300382B091A93042E04DF02DD04188CC3002705183C3820CBDC041A837FFF26C0
S123DD800486012015CEC310A609814027158FC300108F8C620026F08602DE0018381809A6
S123DDA07EDE6B3C1838DE02EE0E1AEF0CCDEF0EDE021AEF0ECDEF0CEC0683000118ED0413
S123DDC0C30001DE00A30018ED06A60318A708EC0418ED00860018A709DC0CC30001DD0CA7
S123DDE018ED0ADC00E306C30008EE068F09DF0018DF0218EE0436A60018A700320918091B
S123DE0083000126F1DE0218081AEF02DE0009DC0CED00183839862020513CEC00DD00CE29
S123DE20C300EC0A1A9300270EEE0E8CC30026F238CC0001ED00399C082604387ECB24182A
S123DE403C8640A7098621B7C6EAEC0C1AEE0E8FCDEF0C1AEF0E183838CC0000ED00398682
S123DE6021B7C6EA391809860320003CDE084D2602861FA70997018621B7C6EA9601812049
S123DE802431CEDEB5A6002708BDDB8825F70820F44FD601C00A25034C20F9CB0A8B30BDD1
S123DEA0DB8825FB178B30BDDB8825FB860ABDDB8825FB38390A52554E54494D45204552A3
S123DEC0522000CE1000DC28E316ED161D237FB610008880B710003BCE1000DC26E31EED91
S123DEE01E1D23F73BCE1000CC07D0E31CED1C1D23EFA62236A7220EDE1408DF142605DE0B
S123DF001208DF127A000A26058621B7C6EA86049D47848027037EDFF09615843F264096E2
S123DF200F8101223A0F4FC6CF9D47DC1E1A8300642D0BCC0000DD1E961C880C971C961C74
S123DF4084082704C6002002C60786029D474FD611C1102502CB30CA809D470E7EDFF0969D
S123DF6039840126037EDFF0960F8102245EDE1A9C16277C088CC2002603CEC110DF1AE675
S123DF8000960F81002634C10A26068601970F205F9611811F27594C9711811126074F375A
S123DFA0C6C09D4733C120250CC17F2208CEE032C0203AE60086029D4720358101260DD717
S123DFC010FCE0209D478602970F2024810A2712CEE020D60F3AEC009D47960F8B02970F82
S123DFE0200E8600970F86019711D610C10A26B5963984042725CE100096224824071C0040
S123E000108B0120031D0010972296234824071C00208B0120031D0020972332B710223BF3
S123E0200001000600CF020000020011495557777FFF202122232425262728292A2B022D16
S123E0402E2F3031323334353637383904053C3D3E3F404142434445464748494A4B4C4D78
S123E0604E4F505152535455565758595A5B5C5D5E5F60616263646566036869066B6C6DB4
S123E0806E6FF0F172737475767778017A7B7C7D7E7F18CE03E8180926FCCE10001F00048A
S123E0A033CC1BE61F00042C83000126F7203937368D56CC00029D47CEE0DD8602E60027F1
S123E0C0059D470820F732BDDCC432BDDCC48602C6299D47CE10001C28204F06CF2A486182
S123E0E06C7465642A2028008D1FCEE0F9BDDD27CE10001D23FB8D163B2D504F574552201C
S123E100474C495443482D20008601979439860E979439CE80004F5FE3008FC300028F8CC2
S109E120FF0226F4393B66
S123BFC0E125E125E125E125E125E125E125E125E125E125E125E125E125E125E125E125FD
S123BFE0DED8DEE5E125E125E125E125E125E092E125E125E125E125E125E125E125C50045
S123FFC0E125E125E125E125E125E125E125E125E125E125E125E125E125E125E125E125BD
S123FFE0DED8DEE5E125E125E125E125E125E092E125E125E125E125E125E125E125C50005
S105FF020000F9
S105FF000251A8
S9030000FC
